 FARCmds

 Timestamp is 54ba6e3f (Sat Jan 17 17:14:23 2015)

 Preferred load address is 0000000180000000

 Start         Length     Name                   Class
 0001:00000000 000001c0H .idata$5                CODE
 0001:000001c0 000005c8H .rdata                  CODE
 0001:00000790 000061efH .text                   CODE
 0001:00006980 000006f8H .xdata                  CODE
 0001:00007078 00000064H .idata$2                CODE
 0001:000070dc 00000014H .idata$3                CODE
 0001:000070f0 000001c0H .idata$4                CODE
 0001:000072b0 000003d8H .idata$6                CODE
 0001:00007690 000000a5H .edata                  CODE
 0002:00000000 00000138H .data                   DATA
 0002:00000140 00001700H .bss                    DATA
 0003:00000000 0000057cH .pdata                  DATA
 0004:00000000 00000058H .rsrc$01                DATA
 0004:00000060 00000378H .rsrc$02                DATA

  Address         Publics by Value              Rva+Base               Lib:Object

 0000:00000000       ___safe_se_handler_table   0000000000000000     <absolute>
 0000:00000000       ___safe_se_handler_count   0000000000000000     <absolute>
 0000:00000000       __ImageBase                0000000180000000     <linker-defined>
 0001:00000000       __imp_RegCloseKey          0000000180001000     advapi32:ADVAPI32.dll
 0001:00000008       __imp_RegQueryValueExW     0000000180001008     advapi32:ADVAPI32.dll
 0001:00000010       __imp_RegOpenKeyExW        0000000180001010     advapi32:ADVAPI32.dll
 0001:00000018       __imp_IsTextUnicode        0000000180001018     advapi32:ADVAPI32.dll
 0001:00000020       \177ADVAPI32_NULL_THUNK_DATA 0000000180001020     advapi32:ADVAPI32.dll
 0001:00000028       __imp_GetConsoleAliasesW   0000000180001028     kernel32:KERNEL32.dll
 0001:00000030       __imp_GetConsoleAliasesLengthW 0000000180001030     kernel32:KERNEL32.dll
 0001:00000038       __imp_lstrcatW             0000000180001038     kernel32:KERNEL32.dll
 0001:00000040       __imp_GetLastError         0000000180001040     kernel32:KERNEL32.dll
 0001:00000048       __imp_GetModuleFileNameW   0000000180001048     kernel32:KERNEL32.dll
 0001:00000050       __imp_CloseHandle          0000000180001050     kernel32:KERNEL32.dll
 0001:00000058       __imp_ReadFile             0000000180001058     kernel32:KERNEL32.dll
 0001:00000060       __imp_CreateFileW          0000000180001060     kernel32:KERNEL32.dll
 0001:00000068       __imp_MultiByteToWideChar  0000000180001068     kernel32:KERNEL32.dll
 0001:00000070       __imp_GetACP               0000000180001070     kernel32:KERNEL32.dll
 0001:00000078       __imp_GetConsoleOutputCP   0000000180001078     kernel32:KERNEL32.dll
 0001:00000080       __imp_SetConsoleTitleW     0000000180001080     kernel32:KERNEL32.dll
 0001:00000088       __imp_GetConsoleWindow     0000000180001088     kernel32:KERNEL32.dll
 0001:00000090       __imp_GetCurrentDirectoryW 0000000180001090     kernel32:KERNEL32.dll
 0001:00000098       __imp_RemoveDirectoryW     0000000180001098     kernel32:KERNEL32.dll
 0001:000000a0       __imp_DeleteFileW          00000001800010a0     kernel32:KERNEL32.dll
 0001:000000a8       __imp_GetFileSize          00000001800010a8     kernel32:KERNEL32.dll
 0001:000000b0       __imp_WriteConsoleW        00000001800010b0     kernel32:KERNEL32.dll
 0001:000000b8       __imp_ExpandEnvironmentStringsW 00000001800010b8     kernel32:KERNEL32.dll
 0001:000000c0       __imp_GetTempFileNameW     00000001800010c0     kernel32:KERNEL32.dll
 0001:000000c8       __imp_CreateDirectoryW     00000001800010c8     kernel32:KERNEL32.dll
 0001:000000d0       __imp_SearchPathW          00000001800010d0     kernel32:KERNEL32.dll
 0001:000000d8       __imp_GetEnvironmentVariableW 00000001800010d8     kernel32:KERNEL32.dll
 0001:000000e0       __imp_WaitForSingleObject  00000001800010e0     kernel32:KERNEL32.dll
 0001:000000e8       __imp_CreateThread         00000001800010e8     kernel32:KERNEL32.dll
 0001:000000f0       __imp_CreateProcessW       00000001800010f0     kernel32:KERNEL32.dll
 0001:000000f8       __imp_SetCurrentDirectoryW 00000001800010f8     kernel32:KERNEL32.dll
 0001:00000100       __imp_SetConsoleMode       0000000180001100     kernel32:KERNEL32.dll
 0001:00000108       __imp_SetConsoleCursorPosition 0000000180001108     kernel32:KERNEL32.dll
 0001:00000110       __imp_GetConsoleScreenBufferInfo 0000000180001110     kernel32:KERNEL32.dll
 0001:00000118       __imp_GetConsoleMode       0000000180001118     kernel32:KERNEL32.dll
 0001:00000120       __imp_GetStdHandle         0000000180001120     kernel32:KERNEL32.dll
 0001:00000128       __imp_HeapFree             0000000180001128     kernel32:KERNEL32.dll
 0001:00000130       __imp_GetProcessHeap       0000000180001130     kernel32:KERNEL32.dll
 0001:00000138       __imp_HeapAlloc            0000000180001138     kernel32:KERNEL32.dll
 0001:00000140       __imp_HeapReAlloc          0000000180001140     kernel32:KERNEL32.dll
 0001:00000148       __imp_GetFileAttributesW   0000000180001148     kernel32:KERNEL32.dll
 0001:00000150       __imp_lstrlenW             0000000180001150     kernel32:KERNEL32.dll
 0001:00000158       __imp_lstrcpyW             0000000180001158     kernel32:KERNEL32.dll
 0001:00000160       __imp_Sleep                0000000180001160     kernel32:KERNEL32.dll
 0001:00000168       __imp_lstrcpynW            0000000180001168     kernel32:KERNEL32.dll
 0001:00000170       \177KERNEL32_NULL_THUNK_DATA 0000000180001170     kernel32:KERNEL32.dll
 0001:00000178       __imp_UuidFromStringW      0000000180001178     rpcrt4:RPCRT4.dll
 0001:00000180       \177RPCRT4_NULL_THUNK_DATA 0000000180001180     rpcrt4:RPCRT4.dll
 0001:00000188       __imp_GetWindowTextW       0000000180001188     user32:USER32.dll
 0001:00000190       __imp_GetWindowTextLengthW 0000000180001190     user32:USER32.dll
 0001:00000198       \177USER32_NULL_THUNK_DATA 0000000180001198     user32:USER32.dll
 0001:000001a0       __imp_CoUninitialize       00000001800011a0     ole32:ole32.dll
 0001:000001a8       __imp_CoCreateInstance     00000001800011a8     ole32:ole32.dll
 0001:000001b0       __imp_CoInitialize         00000001800011b0     ole32:ole32.dll
 0001:000001b8       \177ole32_NULL_THUNK_DATA  00000001800011b8     ole32:ole32.dll
 0001:000001c0       ??_C@_1BE@KBOCGMKN@?$AAS?$AAe?$AAp?$AAa?$AAr?$AAa?$AAt?$AAo?$AAr?$AA?$AA@ 00000001800011c0     FARCmds.obj
 0001:000001d8       ??_C@_1BI@BKNCFIOG@?$AAM?$AAa?$AAx?$AAD?$AAa?$AAt?$AAa?$AAS?$AAi?$AAz?$AAe?$AA?$AA@ 00000001800011d8     FARCmds.obj
 0001:000001f0       ??_C@_1BK@LOJIPNKK@?$AAE?$AAd?$AAi?$AAt?$AAN?$AAe?$AAw?$AAF?$AAi?$AAl?$AAe?$AAs?$AA?$AA@ 00000001800011f0     FARCmds.obj
 0001:00000210       ??_C@_1BM@BMDAMABJ@?$AAV?$AAi?$AAe?$AAw?$AAZ?$AAe?$AAr?$AAo?$AAF?$AAi?$AAl?$AAe?$AAs?$AA?$AA@ 0000000180001210     FARCmds.obj
 0001:00000230       ??_C@_1BE@EKEFMMPP@?$AAC?$AAa?$AAt?$AAc?$AAh?$AAM?$AAo?$AAd?$AAe?$AA?$AA@ 0000000180001230     FARCmds.obj
 0001:00000248       ??_C@_1BM@IEHCKIMD@?$AAS?$AAh?$AAo?$AAw?$AAC?$AAm?$AAd?$AAO?$AAu?$AAt?$AAp?$AAu?$AAt?$AA?$AA@ 0000000180001248     FARCmds.obj
 0001:00000268       MainGuid                   0000000180001268     FARCmds.obj
 0001:00000278       ConfigMenuGuid             0000000180001278     FARCmds.obj
 0001:00000288       DialogGuid                 0000000180001288     FARCmds.obj
 0001:00000298       ??_C@_1DE@BGKMIKPD@?$AAE?$AAu?$AAg?$AAe?$AAn?$AAe?$AA?5?$AAR?$AAo?$AAs?$AAh?$AAa?$AAl?$AA?5?$AA?$CG?$AA?5?$AAF?$AAa?$AAr?$AA?5?$AAG?$AAr?$AAo?$AAu?$AAp?$AA?$AA@ 0000000180001298     FARCmds.obj
 0001:000002d0       ??_C@_1EI@IHKPBHMH@?$AAF?$AAA?$AAR?$AA?5?$AAC?$AAo?$AAm?$AAm?$AAa?$AAn?$AAd?$AAs?$AA?5?$AAP?$AAl?$AAu?$AAg?$AAi?$AAn?$AA?5?$AAf?$AAo?$AAr?$AA?5?$AAF?$AAa?$AAr?$AA?5?$AAM?$AAa?$AAn?$AAa@ 00000001800012d0     FARCmds.obj
 0001:00000318       ??_C@_1BA@LGNBLCFH@?$AAF?$AAA?$AAR?$AAC?$AAm?$AAd?$AAs?$AA?$AA@ 0000000180001318     FARCmds.obj
 0001:00000328       ??_C@_13HOIJIPNN@?$AA?5?$AA?$AA@ 0000000180001328     FARCmds.obj
 0001:00000330       ??_C@_1GC@PBJAIBOO@?$AAv?$AAi?$AAe?$AAw?$AA?3?$AAe?$AAd?$AAi?$AAt?$AA?3?$AAg?$AAo?$AAt?$AAo?$AA?3?$AAc?$AAl?$AAi?$AAp?$AA?3?$AAw?$AAh?$AAe?$AAr?$AAe?$AAi?$AAs?$AA?3?$AAl?$AAi?$AAn?$AAk@ 0000000180001330     FARCmds.obj
 0001:00000398       ??_7?$DialogItemBinding@UFarDialogItem@@@@6B@ 0000000180001398     FARCmds.obj
 0001:000003b0       ??_7?$DialogBuilderBase@UFarDialogItem@@@@6B@ 00000001800013b0     FARCmds.obj
 0001:000003f8       ??_C@_15EFLNJKHH@?$AA?$CF?$AAu?$AA?$AA@ 00000001800013f8     FARCmds.obj
 0001:00000400       ??_7PluginUIntEditFieldBinding@@6B@ 0000000180001400     FARCmds.obj
 0001:00000410       ??_7PluginDialogBuilder@@6B@ 0000000180001410     FARCmds.obj
 0001:00000458       ??_7PluginCheckBoxBinding@@6B@ 0000000180001458     FARCmds.obj
 0001:00000468       ??_7PluginRadioButtonBinding@@6B@ 0000000180001468     FARCmds.obj
 0001:00000478       ??_7PluginIntEditFieldBinding@@6B@ 0000000180001478     FARCmds.obj
 0001:00000488       ??_C@_11LOCGONAA@?$AA?$AA@ 0000000180001488     FARCmds.obj
 0001:00000490       ??_C@_1O@BJPKKLLM@?$AAC?$AAo?$AAn?$AAf?$AAi?$AAg?$AA?$AA@ 0000000180001490     FARCmds.obj
 0001:000004a0       ??_C@_15BNIPFGCG@?$AA$?$AA?$CK?$AA?$AA@ 00000001800014a0     Mix.obj
 0001:000004a8       ??_C@_1BE@EKCMLKPN@?$AA?$CF?$AAC?$AAO?$AAM?$AAS?$AAP?$AAE?$AAC?$AA?$CF?$AA?$AA@ 00000001800014a8     Mix.obj
 0001:000004c0       ??_C@_0BC@KFCLBIA@?$AB?$BE?$AC?$AA?$AA?$AA?$AA?$AA?$MA?$AA?$AA?$AA?$AA?$AA?$AAF?$JL?$AA@ 00000001800014c0     Mix.obj
 0001:000004d4       ??_C@_13FPGAJAPJ@?$AA?2?$AA?$AA@ 00000001800014d4     OpenCmd.obj
 0001:000004d8       ??_C@_1BE@BNONMOPA@?$AA?2?$AA?2?$AA?4?$AA?2?$AAc?$AAd?$AAr?$AAo?$AAm?$AA?$AA@ 00000001800014d8     OpenCmd.obj
 0001:000004f0       ??_C@_1CE@JKDBMIKG@?$AA?2?$AA?2?$AA?4?$AA?2?$AAP?$AAh?$AAy?$AAs?$AAi?$AAc?$AAa?$AAl?$AAD?$AAr?$AAi?$AAv?$AAe?$AA?$AA@ 00000001800014f0     OpenCmd.obj
 0001:00000518       ??_C@_19BKJMDJK@?$AA?2?$AA?2?$AA?4?$AA?2?$AA?$AA@ 0000000180001518     OpenCmd.obj
 0001:00000528       ??_C@_17IJMNDCL@?$AA?$CF?$AAl?$AAu?$AA?$AA@ 0000000180001528     OpenCmd.obj
 0001:00000530       ??_C@_1BA@EIPEFBMB@?$AA?$CF?$AAl?$AAu?$AA?1?$AA?$CF?$AAl?$AAu?$AA?$AA@ 0000000180001530     OpenCmd.obj
 0001:00000550       ??_C@_1GK@PPEHOOAL@?$AAS?$AAO?$AAF?$AAT?$AAW?$AAA?$AAR?$AAE?$AA?2?$AAM?$AAi?$AAc?$AAr?$AAo?$AAs?$AAo?$AAf?$AAt?$AA?2?$AAW?$AAi?$AAn?$AAd?$AAo?$AAw?$AAs?$AA?2?$AAC?$AAu?$AAr?$AAr?$AAe@ 0000000180001550     OpenCmd.obj
 0001:000005bc       ??_C@_13PJJBFPED@?$AA?$DL?$AA?$AA@ 00000001800015bc     OpenCmd.obj
 0001:000005c0       ??_C@_1BA@HAHEJCII@?$AAP?$AAA?$AAT?$AAH?$AAE?$AAX?$AAT?$AA?$AA@ 00000001800015c0     OpenCmd.obj
 0001:000005d0       ??_C@_19IJOJOJIB@?$AAP?$AAA?$AAT?$AAH?$AA?$AA@ 00000001800015d0     OpenCmd.obj
 0001:000005e0       ??_C@_1BA@IBNPAI@?$AAF?$AAA?$AAR?$AAH?$AAO?$AAM?$AAE?$AA?$AA@ 00000001800015e0     OpenCmd.obj
 0001:000005f0       ??_C@_15GBHPEJPD@?$AA?1?$AAS?$AA?$AA@ 00000001800015f0     OpenCmd.obj
 0001:000005f8       ??_C@_15MDAMMGLB@?$AA?1?$AAN?$AA?$AA@ 00000001800015f8     OpenCmd.obj
 0001:00000600       ??_C@_19JMGCACDF@?$AA?1?$AAM?$AAS?$AAG?$AA?$AA@ 0000000180001600     OpenCmd.obj
 0001:0000060c       ??_C@_13NEIAEHFG@?$AA?$CC?$AA?$AA@ 000000018000160c     OpenCmd.obj
 0001:00000610       ??_C@_1BM@MDBPDFDA@?$AA?$CF?$AAC?$AAO?$AAM?$AAS?$AAP?$AAE?$AAC?$AA?$CF?$AA?5?$AA?1?$AAc?$AA?5?$AA?$AA@ 0000000180001610     OpenCmd.obj
 0001:00000630       ??_C@_1BC@ENICKDH@?$AAC?$AAo?$AAn?$AAt?$AAe?$AAn?$AAt?$AAs?$AA?$AA@ 0000000180001630     OpenCmd.obj
 0001:00000648       ??_C@_17KKFGGCGH@?$AAR?$AAU?$AAN?$AA?$AA@ 0000000180001648     OpenCmd.obj
 0001:00000650       ??_C@_17NMIMIGP@?$AAR?$AAu?$AAn?$AA?$AA@ 0000000180001650     OpenCmd.obj
 0001:00000658       ??_C@_19JHOCBEIE@?$AAV?$AAI?$AAE?$AAW?$AA?$AA@ 0000000180001658     OpenCmd.obj
 0001:00000668       ??_C@_19MJAKNMNK@?$AAV?$AAi?$AAe?$AAw?$AA?$AA@ 0000000180001668     OpenCmd.obj
 0001:00000678       ??_C@_19PEJAKIIO@?$AAC?$AAL?$AAI?$AAP?$AA?$AA@ 0000000180001678     OpenCmd.obj
 0001:00000688       ??_C@_19KKHIGANA@?$AAC?$AAl?$AAi?$AAp?$AA?$AA@ 0000000180001688     OpenCmd.obj
 0001:00000698       ??_C@_1BA@NBLHMMII@?$AAW?$AAH?$AAE?$AAR?$AAE?$AAI?$AAS?$AA?$AA@ 0000000180001698     OpenCmd.obj
 0001:000006a8       ??_C@_1BA@BCPLKBBA@?$AAW?$AAh?$AAe?$AAr?$AAe?$AAI?$AAs?$AA?$AA@ 00000001800016a8     OpenCmd.obj
 0001:000006b8       ??_C@_19KFAJFECL@?$AAE?$AAD?$AAI?$AAT?$AA?$AA@ 00000001800016b8     OpenCmd.obj
 0001:000006c8       ??_C@_19PLOBJMHF@?$AAE?$AAd?$AAi?$AAt?$AA?$AA@ 00000001800016c8     OpenCmd.obj
 0001:000006d8       ??_C@_19MEMGFJJL@?$AAG?$AAO?$AAT?$AAO?$AA?$AA@ 00000001800016d8     OpenCmd.obj
 0001:000006e8       ??_C@_19JKCOJBMF@?$AAG?$AAo?$AAt?$AAo?$AA?$AA@ 00000001800016e8     OpenCmd.obj
 0001:000006f8       ??_C@_19NHGGBNEB@?$AAL?$AAI?$AAN?$AAK?$AA?$AA@ 00000001800016f8     OpenCmd.obj
 0001:00000708       ??_C@_19IJIONFBP@?$AAL?$AAi?$AAn?$AAk?$AA?$AA@ 0000000180001708     OpenCmd.obj
 0001:00000718       ??_C@_19LIDMLGEF@?$AAL?$AAO?$AAA?$AAD?$AA?$AA@ 0000000180001718     OpenCmd.obj
 0001:00000728       ??_C@_19OGNEHOBL@?$AAL?$AAo?$AAa?$AAd?$AA?$AA@ 0000000180001728     OpenCmd.obj
 0001:00000738       ??_C@_1O@PAPHGGOK@?$AAU?$AAN?$AAL?$AAO?$AAA?$AAD?$AA?$AA@ 0000000180001738     OpenCmd.obj
 0001:00000748       ??_C@_1O@PJHDHGJM@?$AAU?$AAn?$AAl?$AAo?$AAa?$AAd?$AA?$AA@ 0000000180001748     OpenCmd.obj
 0001:00000758       IID_IShellLinkW            0000000180001758     shell32:shguid.obj
 0001:00000768       IID_IPersistFile           0000000180001768     uuid:objidl_i.obj
 0001:00000778       CLSID_ShellLink            0000000180001778     uuid:shguids2.obj
 0001:000007a0       _alloca_probe              00000001800017a0     chkstk.obj
 0001:000007a0       __chkstk                   00000001800017a0 f   chkstk.obj
 0001:000007f0       ?GetLangString@PluginDialogBuilder@@MEAAPEB_WH@Z 00000001800017f0 f i FARCmds.obj
 0001:00000800       GetGlobalInfoW             0000000180001800 f   FARCmds.obj
 0001:00000880       SetStartupInfoW            0000000180001880 f   FARCmds.obj
 0001:00000b00       OpenW                      0000000180001b00 f   FARCmds.obj
 0001:00000df0       GetPluginInfoW             0000000180001df0 f   FARCmds.obj
 0001:00000e50       ?InitDialogItem@?$DialogBuilderBase@UFarDialogItem@@@@MEAAXPEAUFarDialogItem@@PEB_W@Z 0000000180001e50 f i FARCmds.obj
 0001:00000e50       ?SaveValue@?$DialogItemBinding@UFarDialogItem@@@@UEAAXPEAUFarDialogItem@@H@Z 0000000180001e50 f i FARCmds.obj
 0001:00000e60       ?TextWidth@?$DialogBuilderBase@UFarDialogItem@@@@MEAAHAEBUFarDialogItem@@@Z 0000000180001e60 f i FARCmds.obj
 0001:00000e70       ?DoShowDialog@?$DialogBuilderBase@UFarDialogItem@@@@MEAA_JXZ 0000000180001e70 f i FARCmds.obj
 0001:00000e80       ??1?$DialogBuilderBase@UFarDialogItem@@@@MEAA@XZ 0000000180001e80 f i FARCmds.obj
 0001:00000f00       ?CreateCheckBoxBinding@?$DialogBuilderBase@UFarDialogItem@@@@MEAAPEAU?$DialogItemBinding@UFarDialogItem@@@@PEAHH@Z 0000000180001f00 f i FARCmds.obj
 0001:00000f00       ?AddUIntEditField@?$DialogBuilderBase@UFarDialogItem@@@@UEAAPEAUFarDialogItem@@PEAIH@Z 0000000180001f00 f i FARCmds.obj
 0001:00000f00       ?CreateRadioButtonBinding@?$DialogBuilderBase@UFarDialogItem@@@@MEAAPEAU?$DialogItemBinding@UFarDialogItem@@@@PEAH@Z 0000000180001f00 f i FARCmds.obj
 0001:00000f00       ?GetLangString@?$DialogBuilderBase@UFarDialogItem@@@@MEAAPEB_WH@Z 0000000180001f00 f i FARCmds.obj
 0001:00000f00       ?AddIntEditField@?$DialogBuilderBase@UFarDialogItem@@@@UEAAPEAUFarDialogItem@@PEAHH@Z 0000000180001f00 f i FARCmds.obj
 0001:00000f10       ??_E?$DialogBuilderBase@UFarDialogItem@@@@MEAAPEAXI@Z 0000000180001f10 f i FARCmds.obj
 0001:00000f10       ??_G?$DialogBuilderBase@UFarDialogItem@@@@MEAAPEAXI@Z 0000000180001f10 f i FARCmds.obj
 0001:00000f40       ?ReallocDialogItems@?$DialogBuilderBase@UFarDialogItem@@@@IEAAXXZ 0000000180001f40 f i FARCmds.obj
 0001:00001060       ?ItemWidth@?$DialogBuilderBase@UFarDialogItem@@@@IEAA_JAEBUFarDialogItem@@@Z 0000000180002060 f i FARCmds.obj
 0001:00001100       ?SaveValues@?$DialogBuilderBase@UFarDialogItem@@@@IEAAXXZ 0000000180002100 f i FARCmds.obj
 0001:000011a0       ?MaxTextWidth@?$DialogBuilderBase@UFarDialogItem@@@@IEAA_JXZ 00000001800021a0 f i FARCmds.obj
 0001:000012c0       ??0PluginUIntEditFieldBinding@@QEAA@AEBUPluginStartupInfo@@PEAPEAXHPEAIH@Z 00000001800022c0 f i FARCmds.obj
 0001:00001380       ?SaveValue@PluginUIntEditFieldBinding@@UEAAXPEAUFarDialogItem@@H@Z 0000000180002380 f i FARCmds.obj
 0001:000013d0       ?InitDialogItem@PluginDialogBuilder@@MEAAXPEAUFarDialogItem@@PEB_W@Z 00000001800023d0 f i FARCmds.obj
 0001:00001400       ?TextWidth@PluginDialogBuilder@@MEAAHAEBUFarDialogItem@@@Z 0000000180002400 f i FARCmds.obj
 0001:00001410       ?DoShowDialog@PluginDialogBuilder@@MEAA_JXZ 0000000180002410 f i FARCmds.obj
 0001:000014c0       ?SaveValue@PluginCheckBoxBinding@@UEAAXPEAUFarDialogItem@@H@Z 00000001800024c0 f i FARCmds.obj
 0001:00001520       ?SaveValue@PluginRadioButtonBinding@@UEAAXPEAUFarDialogItem@@H@Z 0000000180002520 f i FARCmds.obj
 0001:00001570       ??0PluginIntEditFieldBinding@@QEAA@AEBUPluginStartupInfo@@PEAPEAXHPEAHH@Z 0000000180002570 f i FARCmds.obj
 0001:00001630       ?SaveValue@PluginIntEditFieldBinding@@UEAAXPEAUFarDialogItem@@H@Z 0000000180002630 f i FARCmds.obj
 0001:00001680       ?CreateCheckBoxBinding@PluginDialogBuilder@@MEAAPEAU?$DialogItemBinding@UFarDialogItem@@@@PEAHH@Z 0000000180002680 f i FARCmds.obj
 0001:00001700       ?CreateRadioButtonBinding@PluginDialogBuilder@@MEAAPEAU?$DialogItemBinding@UFarDialogItem@@@@PEAH@Z 0000000180002700 f i FARCmds.obj
 0001:00001770       ??_GPluginDialogBuilder@@UEAAPEAXI@Z 0000000180002770 f i FARCmds.obj
 0001:00001770       ??_EPluginDialogBuilder@@UEAAPEAXI@Z 0000000180002770 f i FARCmds.obj
 0001:000017c0       ?AddDialogItem@?$DialogBuilderBase@UFarDialogItem@@@@IEAAPEAUFarDialogItem@@W4FARDIALOGITEMTYPES@@PEB_W@Z 00000001800027c0 f i FARCmds.obj
 0001:00001850       ?AddTextBefore@?$DialogBuilderBase@UFarDialogItem@@@@QEAAPEAUFarDialogItem@@PEAU2@H@Z 0000000180002850 f i FARCmds.obj
 0001:00001950       ?AddButtons@?$DialogBuilderBase@UFarDialogItem@@@@QEAAXHPEBHHH@Z 0000000180002950 f i FARCmds.obj
 0001:00001aa0       ?UpdateBorderSize@?$DialogBuilderBase@UFarDialogItem@@@@IEAAXXZ 0000000180002aa0 f i FARCmds.obj
 0001:00001b60       ??_EPluginCheckBoxBinding@@UEAAPEAXI@Z 0000000180002b60 f i FARCmds.obj
 0001:00001b60       ??_GPluginUIntEditFieldBinding@@UEAAPEAXI@Z 0000000180002b60 f i FARCmds.obj
 0001:00001b60       ??_E?$DialogItemBinding@UFarDialogItem@@@@UEAAPEAXI@Z 0000000180002b60 f i FARCmds.obj
 0001:00001b60       ??_G?$DialogItemBinding@UFarDialogItem@@@@UEAAPEAXI@Z 0000000180002b60 f i FARCmds.obj
 0001:00001b60       ??_EPluginUIntEditFieldBinding@@UEAAPEAXI@Z 0000000180002b60 f i FARCmds.obj
 0001:00001b60       ??_EPluginIntEditFieldBinding@@UEAAPEAXI@Z 0000000180002b60 f i FARCmds.obj
 0001:00001b60       ??_GPluginCheckBoxBinding@@UEAAPEAXI@Z 0000000180002b60 f i FARCmds.obj
 0001:00001b60       ??_GPluginIntEditFieldBinding@@UEAAPEAXI@Z 0000000180002b60 f i FARCmds.obj
 0001:00001b60       ??_GPluginRadioButtonBinding@@UEAAPEAXI@Z 0000000180002b60 f i FARCmds.obj
 0001:00001b60       ??_EPluginRadioButtonBinding@@UEAAPEAXI@Z 0000000180002b60 f i FARCmds.obj
 0001:00001b90       ?AddIntEditField@PluginDialogBuilder@@UEAAPEAUFarDialogItem@@PEAHH@Z 0000000180002b90 f i FARCmds.obj
 0001:00001ca0       ?AddUIntEditField@PluginDialogBuilder@@UEAAPEAUFarDialogItem@@PEAIH@Z 0000000180002ca0 f i FARCmds.obj
 0001:00001db0       ConfigureW                 0000000180002db0 f   FARCmds.obj
 0001:00002a70       ?GetMsg@@YAPEB_WH@Z        0000000180003a70 f   Mix.obj
 0001:00002a90       ?ExpandEnv@@YAPEA_WPEB_WPEAK@Z 0000000180003a90 f   Mix.obj
 0001:00002b10       ?GetInt@@YAHPEB_WPEA_W@Z   0000000180003b10 f   Mix.obj
 0001:00002c00       ?PartCmdLine@@YAHPEB_WPEAPEA_W1@Z 0000000180003c00 f   Mix.obj
 0001:00002f00       ?ProcessOSAliases@@YAPEA_WPEB_W@Z 0000000180003f00 f   Mix.obj
 0001:00003260       ?GetShellLinkPath@@YAPEA_WPEB_W@Z 0000000180004260 f   Mix.obj
 0001:00003580       ?StrToGuid@@YA_NPEB_WPEAU_GUID@@@Z 0000000180004580 f   Mix.obj
 0001:000035a0       ?IsTextUTF8@@YA_NPEBD_K@Z  00000001800045a0 f   Mix.obj
 0001:00003640       ?GetCPBuffer@@YAIPEBX_KPEA_K@Z 0000000180004640 f   Mix.obj
 0001:00003750       ?ConvertBuffer@@YAPEA_WPEA_W_KHAEA_KPEA_N@Z 0000000180004750 f   Mix.obj
 0001:000038b0       ??0ConsoleTitle@@QEAA@PEB_W@Z 00000001800048b0 f i OpenCmd.obj
 0001:00003960       ??0MakeVETitle@@QEAA@PEB_W0@Z 0000000180004960 f i OpenCmd.obj
 0001:00003c10       ?isDevice@@YA_NPEB_W0@Z    0000000180004c10 f i OpenCmd.obj
 0001:00004060       ?ThreadWhatUpdateScreen@@YAKPEAX@Z 0000000180005060 f   OpenCmd.obj
 0001:00004740       ?__proc_Load@@YAPEA_WHPEA_W@Z 0000000180005740 f   OpenCmd.obj
 0001:000047b0       ?__proc_Unload@@YAPEA_WHPEA_W@Z 00000001800057b0 f   OpenCmd.obj
 0001:000048b0       ?__proc_Goto@@YAPEA_WHPEA_W@Z 00000001800058b0 f   OpenCmd.obj
 0001:00004930       ?__proc_WhereIs@@YAPEA_WHPEA_W_N@Z 0000000180005930 f   OpenCmd.obj
 0001:00004fc0       ?__proc_Link@@YA_NHPEA_W@Z 0000000180005fc0 f   OpenCmd.obj
 0001:00005490       ?OpenFromCommandLine@@YAPEA_WPEB_W@Z 0000000180006490 f   OpenCmd.obj
 0001:00006600       memcpy                     0000000180007600 f   libCRT64:memcpy.obj
 0001:00006630       free                       0000000180007630 f   libCRT64:free.obj
 0001:00006660       malloc                     0000000180007660 f   libCRT64:malloc.obj
 0001:00006690       ??_V@YAXPEAX@Z             0000000180007690 f   libCRT64:delete_array.obj
 0001:000066a0       ??_U@YAPEAX_K@Z            00000001800076a0 f   libCRT64:new_array.obj
 0001:000066b0       memset                     00000001800076b0 f   libCRT64:memset.obj
 0001:000066e0       ??3@YAXPEAX@Z              00000001800076e0 f   libCRT64:delete.obj
 0001:000066f0       ??2@YAPEAX_K@Z             00000001800076f0 f   libCRT64:new.obj
 0001:00006700       wcschr                     0000000180007700 f   libCRT64:strchr.obj
 0001:00006720       wcsstr                     0000000180007720 f   libCRT64:strstr.obj
 0001:00006790       memmove                    0000000180007790 f   libCRT64:memmove.obj
 0001:000067f0       _memicmp                   00000001800077f0 f   libCRT64:memicmp.obj
 0001:00006860       memcmp                     0000000180007860 f   libCRT64:memcmp.obj
 0001:00006890       realloc                    0000000180007890 f   libCRT64:realloc.obj
 0001:00006920       swab                       0000000180007920 f   libCRT64:swab.obj
 0001:00007078       __IMPORT_DESCRIPTOR_KERNEL32 0000000180008078     kernel32:KERNEL32.dll
 0001:0000708c       __IMPORT_DESCRIPTOR_USER32 000000018000808c     user32:USER32.dll
 0001:000070a0       __IMPORT_DESCRIPTOR_ADVAPI32 00000001800080a0     advapi32:ADVAPI32.dll
 0001:000070b4       __IMPORT_DESCRIPTOR_ole32  00000001800080b4     ole32:ole32.dll
 0001:000070c8       __IMPORT_DESCRIPTOR_RPCRT4 00000001800080c8     rpcrt4:RPCRT4.dll
 0001:000070dc       __NULL_IMPORT_DESCRIPTOR   00000001800080dc     kernel32:KERNEL32.dll
 0002:00000000       ?OptName@@3UOptionsName@@A 0000000180009000     FARCmds.obj
 0002:00000140       ?Info@@3UPluginStartupInfo@@A 0000000180009140     FARCmds.obj
 0002:00000250       ?FSF@@3UFarStandardFunctions@@A 0000000180009250     FARCmds.obj
 0002:000003c8       ?Opt@@3UOptions@@A         00000001800093c8     FARCmds.obj

 entry point at        0000:00000000

 Static symbols

 0001:00002dc0       ?GetAlias@@YAPEA_WPEB_W0@Z 0000000180003dc0 f   Mix.obj
 0001:00003a00       ?getCurrDir@@YAPEA_W_N@Z   0000000180004a00 f   OpenCmd.obj
 0001:00003aa0       ?killTemp@@YAXPEA_W@Z      0000000180004aa0 f   OpenCmd.obj
 0001:00003ae0       ?createFile@@YAPEAXPEA_WH@Z 0000000180004ae0 f   OpenCmd.obj
 0001:00003b90       ?createFileStream@@YAXPEB_WPEAXPEAUTShowOutputStreamData@@1@Z 0000000180004b90 f   OpenCmd.obj
 0001:00003ca0       ?validForView@@YA_NPEB_W_N1@Z 0000000180004ca0 f   OpenCmd.obj
 0001:00003f60       ?showPartOfOutput@@YAKPEAUTShowOutputStreamData@@_N@Z 0000000180004f60 f   OpenCmd.obj
 0001:00004230       ?MakeTempNames@@YA_NPEAPEA_W0@Z 0000000180005230 f   OpenCmd.obj
 0001:000043f0       ?loadFile@@YAPEA_WPEB_WKHAEA_KAEA_N@Z 00000001800053f0 f   OpenCmd.obj
 0001:00004610       ?__getContent@@YAPEA_WHPEA_W@Z 0000000180005610 f   OpenCmd.obj
 0001:00005250       ?MakeExecuteString@@YAPEB_WPEB_W@Z 0000000180006250 f   OpenCmd.obj
